:0A00000075817F7401F58F02000E78
:10000B0002023FC229C2287400900010F090001128
:10001B00F0900012F0900013F0900014F074009028
:10002B000016F07401900017F07402900018F07431
:10003B0003900019F0740490001AF0740590001BE3
:10004B00F0740690001CF0740790001DF07408907B
:10005B00001EF0740990001FF0740A900020F074D9
:10006B000B900021F07400900031F0900032F09072
:10007B000033F0900034F0900035F0740290002FB4
:10008B00F07402900030F090003679FF7400F0A30A
:10009B00D9FA90013579FF7400F0A3D9FA900236A2
:1000AB0079FF7400F0A3D9FA90033579CD7400F081
:1000BB00A3D9FA120EBB7563FF7564FF7565FF75E7
:1000CB00460075470075700075670075710075689F
:1000DB0000C208C2097540007541007542007543A6
:1000EB0000754C00754D00756F027548FF75490A18
:1000FB0085483C85493D754A7F754B01854A44854A
:10010B004B45755500D226C2C175A012C2B1C2B300
:10011B00C2B4C2B5C2B6C281C2B2C2841206A212A6
:10012B0006C11206E01206FF12081675597F755AA2
:10013B007F755B7F755D00755E00755F001201EF6B
:10014B0012059D1205F81221637572007573017506
:10015B0071001216B1121F01121F0CD20FD22CC23A
:10016B002E1223621208161223F4122520121F01DD
:10017B00121F0C1208B9120B0A120ED812152412E8
:10018B00153C121CBC121CA112239702016C85603A
:10019B0090C2A7C2C0D2C022856190D2A7C2C0D2E2
:1001AB00C022C285C281C2B2C284E56379081392B0
:1001BB0083C285D285D9F7D2810000C281E56479EB
:1001CB0008139283C285D285D9F7D2B20000C2B28E
:1001DB00E5657908139283C285D285D9F7D284005D
:1001EB0000C28422758790758922758DFC758BFCF6
:1001FB00759850C299C298758C38758A38753906BE
:10020B00753A04753B0590FF9C8582CA8583CB8527
:10021B0082CC8583CDC200C201D28CD2A9D2AF22AF
:10022B00783279320000D9FCD8F822780A790FD9C4
:10023B00FED8FA22C2AFC0E0C0D0E5F0C0E0E58244
:10024B00C0E0E583C0E0E574C0E0E8C0E0E9C0E0F1
:10025B00EAC0E0EBC0E01206E01224CC1224E0125C
:10026B0011B5D544107544FFD5450A854A44854BD5
:10027B0045D223D22712240E122445121AD112244E
:10028B00241203EB1204491224F4122464D53920EE
:10029B00753906B20330030912071E12068A0202D1
:1002AB00AF1201ADD53A09753A041201991201A3A7
:1002BB00D0E0FBD0E0FAD0E0F9D0E0F8D0E0F57474
:1002CB00D0E0F583D0E0F582D0E0F5F0D0D0D0E0EF
:1002DB00D2AF32E54FB4021130240ED287C2820561
:1002EB004DD2A2121F3E02202322E55575F00124A8
:1002FB001084E5F0B40014E54FB400067556800287
:10030B00037BB4020675568002037B22E55575F01C
:10031B0001241084E5F0B4000BE54FB400067556CC
:10032B005002037B22E55575F002241084E5F0B4EE
:10033B00000BE54FB4000675562202037B22E555F0
:10034B0075F004241084E5F0B4000BE54FB40006FF
:10035B0075561002037B22E55575F008241084E5D1
:10036B00F0B4000BE54FB4000675560702037B2271
:0F037B00200C0C302409D2B6C280D2041211D447
:10038A00D21B85525022E55A75F01E84B40403022A
:10039A000362B40503020349B40603020330B40737
:1003AA0003020317B4080302031722E559B40F0323
:1003BA000203BF500574010203CDC3940F8556F0A2
:1003CA00842401F55222E559B40F030203DA5005D9
:1003DA0074010203E8C3940F8556F0842401F5538F
:1003EA0022D53C03020418D53C03020418D53C0369
:1003FA00020418D53C03020418D53C03020418D59C
:10040A003C03020418D53C03020418D53C0DD53D23
:10041A000A85483C85493D054FD201300120120228
:10042A00DE301B0FD5500CC21B202007302404C21B
:10043A00B6D280121D451203901203B5C20122D50D
:10044A003E0302046AD53E0302046AD53E0302044F
:10045A006AD53E0302046AD53E0302046AD53E0DFC
:10046A00D53F0A85483E85493F054ED20030000BEC
:10047A0012048612057E1203D0C20022201A01221B
:10048A00D5500CC21A202007302404C2B6D28022CA
:10049A00E55575F002241084E5F0B40014E54EB475
:1004AA000006755680020569B40214755680020565
:1004BA0069B4010BE54EB40106755680020569223E
:1004CA00E55575F004241084E5F0B4010BE54EB44B
:1004DA000022755678020569B4020BE54EB4011480
:1004EA00755678020569B4030BE54EB402067556D3
:1004FA007802056922E55575F008241084E5F0B400
:10050A00010BE54EB40022755630020569B4030B9F
:10051A00E54EB40214755630020569B4060BE54E71
:10052A00B4010675563002056922E55575F01024A6
:10053A001084E5F0B4010BE54EB40022755615029D
:10054A000569B4060BE54EB4011475561502056922
:10055A00B40B0BE54EB40206755615020569222046
:10056A000C0C302409D2B6C280D2041211D4D21A89
:10057A0085535022E55A75F01E84B400030204CA5A
:10058A00B401030204CAB402030204FFB40303025F
:10059A000534227563F71202367563DF1202367567
:1005AA0063FF7564F71202367564FD1202367564CC
:1005BA00FF7565DF1202367565FD12023675657FB5
:1005CA001202367565FF75637F1202367563FD1276
:1005DA0002367563FF7564DF12023675647F120294
:1005EA00367564FF7565F71202367565FF22756305
:1005FA00F31202367563CF1202367563FF7564F320
:10060A001202367564FC1202367564FF7565CF12E4
:10061A0002367565FC12023675653F12023675653B
:10062A00FF75633F1202367563FC1202367563FF6B
:10063A007564CF12023675643F1202367564FF750F
:10064A0065F31202367565FF227563001201AD75F6
:10065A0063001201AD7563001201AD756355120195
:0F066A00AD7563001201AD7563001201AD7563CC
:10067900001201AD7565551201AD7564001201AD29
:1006890022E546B4000505460206A2B40105054661
:100699000206C17546000206FF74FE79083392838B
:1006A900D285C285D9F7C2B7D2B77908A2A133D208
:1006B900A6C2A6D9F7F5692274FD7908339283D2C7
:1006C90085C285D9F7C2B7D2B77908A2A133D2A614
:1006D900C2A6D9F7F56A2274FB7908339283D285C9
:1006E900C285D9F7C2B7D2B77908A2A133D2A6C2B7
:1006F900A6D9F7F56B2274F77908339283D285C2AC
:1007090085D9F7C2B7D2B77908A2A133D2A6C2A6B2
:10071900D9F7F56C22E547B40005054702074EB441
:100729000105054702076CB40205054702078EB4A7
:10073900030505470207B0B4040505470207DA7542
:1007490047000207F8C2A3C286C2B0D2A57914D95C
:10075900FEC2A57908C2A6D2A6A2A433D9F7C2A619
:10076900F55D22D2A3C286C2B0D2A57914D9FEC240
:10077900A57908C2A6D2A6A2A433D9F7C2A6302861
:100789000122F55922C2A3D286C2B0D2A57914D9C1
:10079900FEC2A57908C2A6D2A6A2A433D9F7C2A6D9
:1007A90030280122F55A22D2A3C286D2B0D2A57925
:1007B90014D9FEC2A57908C2A6D2A6A2A433D9F734
:1007C900C2A63028030207D3F55B30290122F55C64
:1007D90022D2A3D286C2B0D2A57914D9FEC2A579F4
:1007E90008C2A6D2A6A2A433D9F7C2A6F55E22C230
:1007F900A3C286D2B0D2A57914D9FEC2A57908C2FE
:10080900A6D2A6A2A433D9F7C2A6F55F2212084040
:1008190012084E12083212085C12086A120878127D
:1008290008861208971208A822E56B30E4012220F5
:10083900E60122756D0022E56B20E4012220E60124
:1008490022756D0122E56B20E4012230E601227553
:100859006D0222E56A30E3012220E50122756E006E
:1008690022E56A20E3012220E50122756E0122E5D5
:100879006A20E3012230E50122756E0222E56C301F
:10088900E6012220E50122740190002FF022E56C97
:1008990020E6012220E50122740290002FF022E5D2
:1008A9006C20E6012230E50122740490002FF02229
:1008B900E56E7017C22EC22DD20F1208D5120A0E7C
:1008C90012093A120B041209E1D22C22302907909D
:1008D9000031E00208E1E55CB478030208EC50035A
:1008E9000208EE747975F01784B4000C756600C2BD
:1008F900B1C2B3C2B5C2B422B4010C756601D2B19A
:10090900C2B3C2B5C2B422B4020C756602C2B1D276
:10091900B3C2B5C2B422B4030C756603C2B1C2B383
:10092900D2B5C2B422756604C2B1C2B3C2B5D2B4DB
:1009390022E56675F030A42567F56022E56AF43092
:10094900E009757001D22A1209EA2230E1097570AD
:1009590000D22A1209EA2230E209757002D22A125B
:1009690009EA2230E609757003D22A1209EA22E55A
:1009790069F430E009757006D22A1209EA2230E1D9
:1009890009757009D22A1209EA2230E20975700A3A
:10099900D22A1209EA2230E309757007D22A12090C
:1009A900EA2230E40975700BD22A1209EA2230E5ED
:1009B90009757008D22A1209EA2230E6097570050C
:1009C900D22A1209EA2230E709757004D22A1209DB
:1009D900EA22C22A1209EA22202A03D2A022C2A0AC
:0E09E90022E570202A05C2E7F56822D2E7F564
:1009F7006822900032E020E707C22AC2E7F570229A
:100A0700D22AC2E7F570223029061209F9020A1D17
:100A1700120945020A1DE570B40110756704120931
:100A27003A75637F7564FF7565FF22B400107567BB
:100A37000012093A7563F77564FF7565FF22B40202
:100A47001075670812093A7563DF7564FF7565FFEE
:100A570022B4031075670C12093A7563FD7564FFBC
:100A67007565FF22B4061075671812093A7563FF9A
:100A77007564DF7565FF22B4091075672412093A9A
:100A87007563FF7564FF7565FD22B40A10756728E5
:100A970012093A7563FF7564FF7565F722B407108D
:100AA70075671C12093A7563FF7564FF7565DF2268
:100AB700B40B1075672C12093A7563FF7564FF75DF
:100AC700657F22B4081075672012093A7563FF75B0
:100AD700647F7565FF22B4051075671412093A75AE
:100AE70063FF7564FD7565FF22B404107567101206
:100AF700093A7563FF7564F77565FF2222E5701281
:100B07000CE422E56E7003D20F22E56DB40212D217
:100B17002CC22EC22D300F05120EAFC20F120CC7FA
:100B270022D20F22E55EB43803020B355003790059
:100B370022B43C03020B405003790122B441030263
:100B47000B4B5003790222B44503020B565003792D
:100B57000322B44A03020B615003790422B44E0303
:100B6700020B6C5003790522B45303020B77500331
:100B7700790622B45703020B825003790722B45C2B
:100B870003020B8D5003790822B46003020B9850BF
:100B970003790922B46503020BA35003790A22B42F
:100BA7006A03020BAE5003790B22790B22120B2B2F
:100BB700E9900033F0120CC2120EAF22900033E01E
:100BC700F574120B2BE9B57403020BEDE55EB43433
:100BD70004120BB4225003020BEDB46B03020BEDAE
:100BE7005004120BB422E56AF430E00E200E51D205
:100BF7000E7901120CC2120EAF2230E10E200E4008
:100C0700D20E7900120CC2120EAF2230E20E200E65
:100C17002FD20E7902120CC2120EAF2230E60E202E
:100C27000E1ED20E7903120CC2120EAF22E569F422
:100C370030E00E200E0AD20E7906120CC2120EAF49
:100C47002230E10E200E70D20E7909120CC2120E5C
:100C5700AF2230E20E200E5FD20E790A120CC212BA
:100C67000EAF2230E30E200E4ED20E7907120CC2C1
:100C7700120EAF2230E40E200E3DD20E790B120C6D
:100C8700C2120EAF2230E50E200E2CD20E790812BA
:100C97000CC2120EAF2230E60E200E1BD20E7905C3
:100CA700120CC2120EAF2230E70E200E0AD20E79B6
:100CB70004120CC2120EAF22C20E2289688970225A
:100CC700302911900032E0C2E7B5700122D20FF54A
:100CD70070020EAF020BC3E570120CE422B4010AD6
:100CE70075637F7564FF7565FF22B4000A7563F746
:100CF7007564FF7565FF22B4020A7563DF7564FFCB
:100D07007565FF22B4030A7563FD7564FF7565FF9A
:100D170022B4060A7563FF7564DF7565FF22B4099F
:100D27000A7563FF7564FF7565FD22B40A0A75636A
:100D3700FF7564FF7565F722B4070A7563FF75646D
:0D0D4700FF7565DF22B40B0A7563FF75644C
:100D5400FF75657F22B4080A7563FF75647F756546
:100D6400FF22B4050A7563FF7564FD7565FF22B43F
:100D7400040A7563FF7564F77565FF2222B4010ADE
:100D840075633F7564FF7565FF22B4000A7563F3EC
:100D94007564FF7565FF22B4020A7563CF7564FF3D
:100DA4007565FF22B4030A7563FC7564FF7565FFFE
:100DB40022B4060A7563FF7564CF7565FF22B40912
:100DC4000A7563FF7564FF7565FC22B40A0A7563CE
:100DD400FF7564FF7565F322B4070A7563FF7564D4
:100DE400FF7565CF22B40B0A7563FF7564FF7565E3
:100DF4003F22B4080A7563FF75643F7565FF22B42A
:100E0400050A7563FF7564FC7565FF22B4040A75F1
:100E140063FF7564F37565FF2222B40109E563C2BB
:100E2400E7D2E6F56322B40009E563C2E3D2E2F552
:100E34006322B40209E563C2E5D2E4F56322B40394
:100E440009E563C2E1D2E0F56322B40609E564C2B0
:100E5400E5D2E4F56422B40909E565C2E1D2E0F51E
:100E64006522B40A09E565C2E3D2E2F56522B40756
:100E740009E565C2E5D2E4F56522B40B09E565C26E
:100E8400E7D2E6F56522B40809E564C2E7D2E6F5DF
:100E94006422B40509E564C2E1D2E0F56422B40435
:100EA40009E564C2E3D2E2F5642222120EBB1210F9
:100EB400FAE570120E1E22790C90002205A2900011
:100EC40016E0A320E70605A2F0A305A2D9F305A224
:100ED4007480F022E56E700122E56DB40116D22C07
:100EE400C22F1216EA1216CD202E09120EF9120F75
:100EF400C3120EBB22E56AF430E00D200D4CD20D76
:100F0400900017E0B2E7F02230E10D200D3CD20D45
:100F1400900016E0B2E7F02230E20D200D2CD20D45
:100F2400900018E0B2E7F02230E60D200D1CD20D3F
:100F3400900019E0B2E7F022E569F430E00D200DED
:100F440009D20D90001CE0B2E7F02230E10D200D33
:100F54006DD20D90001FE0B2E7F02230E20D200DBB
:100F64005DD20D900020E0B2E7F02230E30D200DB9
:100F74004DD20D90001DE0B2E7F02230E40D200DBB
:100F84003DD20D900021E0B2E7F02230E50D200DB6
:100F94002DD20D90001EE0B2E7F02230E60D200DB8
:100FA4001DD20D90001BE0B2E7F02230E70D200DBA
:100FB4000DD20D90001AE0B2E7F022C20D22229069
:100FC4000017E020E70BE563C2E7C2E6F563020F12
:100FD400DDE563D2E7D2E6F563900016E020E70B87
:100FE400E563C2E3C2E2F563020FF7E563D2E3D23D
:100FF400E2F563900018E020E70BE563C2E5C2E484
:10100400F563021011E563D2E5D2E4F563900019AB
:10101400E020E70BE563C2E1C2E0F56302102BE5D3
:1010240063D2E1D2E0F56390001CE020E70BE564B5
:10103400C2E5C2E4F564021045E564D2E5D2E4F504
:101044006490001FE020E70BE565C2E1C2E0F565AE
:1010540002105FE565D2E1D2E0F565900020E02062
:0A106400E70BE565C2E3C2E2F565A3
:10106E00021079E565D2E3D2E2F56590001DE0202D
:10107E00E70BE565C2E5C2E4F565021093E565D2BE
:10108E00E5D2E4F565900021E020E70BE565C2E7C7
:10109E00C2E6F5650210ADE565D2E7D2E6F56590DC
:1010AE00001EE020E70BE564C2E7C2E6F56402101D
:1010BE00C7E564D2E7D2E6F56490001BE020E70BAB
:1010CE00E564C2E1C2E0F5640210E1E564D2E1D26A
:1010DE00E0F56490001AE020E709E564C2E3C2E29D
:1010EE00F56422E564D2E3D2E2F564227563FF75FE
:1010FE0064FF7565FF900022E0FAE0F92570C39A4F
:10110E00B40C03021119500302111CC3940C1211DA
:10111E0025A3E930E7E422B40109E563C2E7C2E69C
:10112E00F56322B40009E563C2E3C2E2F56322B4BB
:10113E000209E563C2E5C2E4F56322B40309E5637F
:10114E00C2E1C2E0F56322B40609E564C2E5C2E479
:10115E00F56422B40909E565C2E1C2E0F56522B481
:10116E000A09E565C2E3C2E2F56522B40709E56541
:10117E00C2E5C2E4F56522B40B09E565C2E7C2E635
:10118E00F56522B40809E564C2E7C2E6F56422B447
:10119E000509E564C2E1C2E0F56422B40408E56421
:1011AE00C2E3C2E2F56422E56EB40110E56B30E5F0
:1011BE0003C22522202505D2251214CB22E56EB4BA
:1011CE0002031214CB2230040DC204202008E56E57
:1011DE00B402031214CB22E55DB402030211EF50E8
:1011EE0003790022B406030211FA5003790122B4E6
:1011FE000A030212055003790222B40F03021210E1
:10120E005003790322B4130302121B5003790422F4
:10121E00B418030212265003790522B41D030212DC
:10122E00315003790622B4210302123C5003790790
:10123E0022B425030212475003790822B42A03026E
:10124E0012525003790922B42E0302125D50037913
:10125E000A22B433030212685003790B22790B224F
:10126E00E55DB437030212785003790022B43C03D3
:10127E000212835003790122B4400302128E5003EE
:10128E00790222B445030212995003790322B4491C
:10129E00030212A45003790422B44E030212AF507B
:1012AE0003790522B452030212BA5003790622B40E
:1012BE0057030212C55003790722B45B030212D002
:1012CE005003790822B460030212DB50037909221D
:1012DE00B464030212E65003790A22B468030212C0
:1012EE00F15003790B22790B22E55DB46D030213E5
:1012FE00015003790022B4710302130C50037901DB
:10130E0022B476030213175003790222B47A030231
:10131E0013225003790322B47E0302132D50037956
:10132E000422B483030213385003790522B48703D1
:10133E000213435003790622B48C0302134E50035A
:10134E00790722B490030213595003790822B495F9
:10135E00030213645003790922B4990302136F50E8
:10136E0003790A22B49E0302137A5003790B227971
:10137E000B22E55DB4A20302138A5003790022B456
:10138E00A7030213955003790122B4AB030213A0F5
:10139E005003790222B4B0030213AB500379032237
:1013AE00B4B4030213B65003790422B4B903021382
:1013BE00C15003790522B4BD030213CC5003790644
:1013CE0022B4C1030213D75003790722B4C6030215
:0E13DE0013E25003790822B4CA030213ED5043
:1013EC0003790922B4CF030213F85003790A22B40B
:1013FC00D4030214035003790B22790B22E55DB45C
:10140C00D8030214135003790022B4DC0302141E17
:10141C005003790122B4E10302142950037902220A
:10142C00B4E5030214345003790322B4EA03021422
:10143C003F5003790422B4EE0302144A5003790599
:10144C0022B4F3030214555003790622B4F70302B5
:10145C0014605003790722B4FC0302146B50037917
:10146C000822B4FE030214765003790922790A2269
:10147C00E55DB4330302148650091211E5897474C6
:10148C0000FB22B46803021497500912126E89747F
:10149C007401FB22B49E030214A850091212F7899E
:1014AC00747402FB22B4D4030214B95009121380D1
:1014BC0089747403FB2212140989747404FB2212BC
:1014CC00147C7A00900022E020E70DB5740302141E
:1014DC00E55006A3FA0214D3EA2570F9BB0424B430
:1014EC000A0302150F401C7A00900022E020E70D41
:1014FC002570B40A06E0FAA30214F840F8EA257045
:10150C00021510E975F004A4F9EB75F030A4FAE9B2
:10151C002AF560EB1208F222E56E700122E56DB43B
:10152C00000DC22EC22D1219D612163712156E22AC
:10153C00E56E700122E56DB401151219D630300F2D
:10154C001216B1120EF9120FC3120EBBC23022B416
:10155C00020F1219D63031091216B1120EAFC23168
:10156C002222202C0122E572120D81E573120E1E2F
:10157C00C22CE56E700122E56DB40006302F03120B
:10158C0016B122E56AF430E114E571C2E0C2E1C2A1
:10159C00E2C2E3F571757200D22CD22F2230E21424
:1015AC00E571D2E0C2E1C2E2C2E3F571757202D21A
:1015BC002CD22F22E569F430E114E571D2E0C2E1BE
:1015CC00D2E2C2E3F571757209D22CD22F2230E32C
:1015DC0014E571C2E0C2E1D2E2C2E3F571757207A3
:1015EC00D22CD22F2230E414E571C2E0D2E1D2E247
:1015FC00C2E3F57175720BD22CD22F2230E614E5B2
:10160C0071D2E0D2E1C2E2C2E3F571757205D22C5F
:10161C00D22F2230E714E571C2E0D2E1C2E2C2E37C
:10162C00F571757204D22CD22F2222E56AF430E0C7
:10163C0014E571C2E4C2E5C2E6C2E7F57175730147
:10164C00D22CD22F2230E614E571D2E4C2E5C2E6E8
:10165C00C2E7F571757303D22CD22F22E569F430F1
:10166C00E014E571C2E4D2E5C2E6C2E7F571757328
:10167C0006D22CD22F2230E514E571D2E4D2E5C289
:10168C00E6C2E7F571757308D22CD22F2230E21422
:10169C00E571C2E4C2E5D2E6C2E7F57175730AD210
:1016AC002CD22F2222E571C2E0C2E1C2E2C2E3C415
:1016BC00B40407122116120EBB22122141120EBBCA
:1016CC0022E56B30E303C22B22202B11D22B202DD1
:1016DC0005D22ED22D22C22E1220E6C22D22202E71
:1016EC000122E571C2E4C2E5D2E6C2E7F571757379
:1016FC000A12158F12156E22900034E0F57412192F
:10170C00D6E9B5740302172EE55FB434041219D66A
:10171C0022500302172EB4540302172E5004121930
:10172C00D62212158F22E55FB4370302173C5007FF
:10173C007401900035F022B43C0302174B5007742F
:10174C0002900035F022B4400302175A500774037C
:0E175C00900035F022B445030217695007745F
:10176A0004900035F022B449030217785007740533
:10177A00900035F022B44E03021787500774069082
:10178A000035F022B45203021796500774079000EE
:10179A0035F02222E55FB457030217A850077401F7
:1017AA00900035F022B45B030217B7500774029019
:1017BA000035F022B460030217C650077403900084
:1017CA0035F022B464030217D5500774049000352B
:1017DA00F022B468030217E450077405900035F04C
:1017EA0022B46D030217F350077406900035F022F5
:1017FA00B4710302180250077407900035F02222D0
:10180A00E55FB4760302181450077401900035F0AE
:10181A0022B47A0302182350077402900035F0228A
:10182A00B47E0302183250077403900035F022B4D4
:10183A00830302184150077404900035F022B487DC
:10184A000302185050077405900035F022B48C0337
:10185A0002185F50077406900035F022B490030214
:10186A00186E50077407900035F02222E55FB49590
:10187A000302188050077401900035F022B49903CE
:10188A0002188F50077402900035F022B49E0302AA
:10189A00189E50077403900035F022B4A203021870
:1018AA00AD50077404900035F022B4A7030218BCA7
:1018BA0050077405900035F022B4AB030218CB50E0
:1018CA00077406900035F022B4B0030218DA500704
:1018DA007407900035F02222E55FB4B4030218ECD5
:1018EA0050077401900035F022B4B9030218FB5076
:1018FA00077402900035F022B4BD0302190A50079A
:10190A007403900035F022B4C10302191950077408
:10191A0004900035F022B4C6030219285007740552
:10192A00900035F022B4CA030219375007740690A2
:10193A000035F022B4CF030219465007740790000D
:10194A0035F02222E55FB4330122500122B452035A
:10195A0002195F5013121732E571C2E4C2E5C2E6FA
:10196A00C2E7F57175730122B4710302197A501333
:10197A0012179EE571D2E4C2E5C2E6C2E7F57175B7
:10198A00730322B49003021995501312180AE571D1
:10199A00C2E4D2E5C2E6C2E7F57175730622B4B0B5
:1019AA00030219B05013121876E571D2E4D2E5C2D7
:1019BA00E6C2E7F571757308221218E2E571C2E40E
:1019CA00C2E5D2E6C2E7F57175730A2212194E9082
:1019DA000034E0F575900035E0B5750EE56E7001DE
:1019EA0022E56DB4000312158F22D22F900035E044
:1019FA00900034F0B40103021A065016E571C2E0F1
:101A0A00C2E1C2E2C2E3F571757200D22CD231D2C0
:101A1A003022B40203021A245016E571D2E0C2E160
:101A2A00C2E2C2E3F571757202D22CD231D23022EF
:101A3A00B40303021A425016E571C2E0D2E1C2E2CF
:101A4A00C2E3F571757204D22CD231D23022B404B9
:101A5A0003021A605016E571D2E0D2E1C2E2C2E393
:101A6A00F571757205D22CD231D23022B405030237
:101A7A001A7E5016E571C2E0C2E1D2E2C2E3F57104
:101A8A00757207D22CD231D23022B40603021A9CC4
:101A9A005016E571D2E0C2E1D2E2C2E3F571757285
:101AAA0009D22CD231D23022B40703021ABA501604
:101ABA00E571C2E0D2E1D2E2C2E3F57175720BD2EE
:101ACA002CD231D230222230231A054C121C6A122F
:0E1ADA001B0D121B46121AF1121B35121C189E
:101AE800121C7E121CE2C22322E54C75F0182460F9
:101AF80084E5F0B40C06202402C28222B40005203A
:101B08002402D28222E54C75F006246084E5F0B404
:101B1800030C202408D287121F3E02202322B4007F
:101B28000B202408C287121F3E02202322E54CB452
:101B3800600B754C00202405C2A2121F1722202416
:101B48000BE54CB4000122B40302D2A222E54C7585
:101B5800F030246084E5F0B40009755708756260B8
:101B6800021C5522E54C75F018246084E5F0B40099
:101B78000975570F756260021C5522E54C75F00C0B
:101B8800246084E5F0B4000975571E756260021C74
:101B98005522E54C75F006246084E5F0B40009751B
:101BA800573C756260021C5522E54C75F0032460B1
:101BB80084E5F0B40009755778756260021C5522F7
:101BC800E54C75F020246084E5F0B4000675570AEA
:101BD800021C5522E54C75F010246084E5F0B40031
:101BE80006755714021C5522E54C75F008246084CC
:101BF800E5F0B40006755728021C5522E54C75F02F
:101C080004246084E5F0B40006755750021C552280
:101C1800E55A75F01E84B40003021C04B4010302E3
:101C28001BF0B40203021BDCB40303021BC8B40498
:101C380003021B55B40503021B6CB40603021B8385
:101C4800B40703021B9AB40803021BB122200C0C30
:101C5800202409D2B6C280D2041211D4D21C8554D1
:101C68005122201C0122D5510CC21C2020072024FF
:101C780004C2B6D28022E559B40F03021C8850056D
:101C88007401021C96C3940F8557F0842401F554FF
:101C9800E557B4800375540122E55975F00484B4FE
:101CA8000005D20CC22022B43F05C20CD22022C2A9
:101CB8000CC22022E55BB4A003021CD0500A1223F8
:101CC8003B75F002A4021CDFB4C803021CDE5006F8
:101CD8001223C6021CDF22F56122E55BB4C80302A9
:101CE8001CEC4032B4FA03021CF4502BE54C75F09E
:101CF80003246084E5F0B4001DE54C75F0602460B1
:101D080084E5F0FAC374609A75F00284F5F07405FE
:101D1800A4202402F56122E54C75F003246084E5D3
:101D2800F0B40018E54C75F060246084E5F075F0B7
:101D38000284F5F07405A4202402F56122E55BB461
:101D4800C803021D4F4019B4FA03021D57501274FC
:101D580020C3954D75F008A4122332302402F56192
:101D680022E54D75F008A4122332302402F56122D1
:101D7800202406E54CFB021DA3E54D75F003A4FBEA
:101D8800021DA320240EE54C75F0038475F002A40F
:101D9800FB021DA3E54D75F002A4FB858232858305
:101DA8003375340075350078328B367537007936DF
:101DB80012224F868208868322E571C2E0C2E1C200
:101DC800E2C2E3C4B40004121DE922B40104121EE5
:101DD8002122B40204121E5922B40304121E9122B5
:101DE80022E571C2E4C2E5C2E6C2E7B40004902568
:101DF8008A22B4010490259622B402049025A222D6
:101E0800B403049025AE22B404049025BA22B40584
:101E1800049025C6229025D222E571C2E4C2E5C20B
:101E2800E6C2E7B400049025DE22B401049025EA56
:101E380022B402049025F622B4030490260222B4A8
:101E4800040490260E22B4050490261A2290262611
:0E1E580022E571C2E4C2E5C2E6C2E7B40004AE
:101E660090263222B4010490263E22B40204902623
:101E76004A22B4030490265622B404049026622211
:101E8600B4050490266E2290267A22E571C2E4C239
:101E9600E5C2E6C2E7B4000490268622B4010490A7
:101EA600269222B4020490269E22B403049026AA07
:101EB60022B404049026B622B405049026C22290C9
:101EC60026CE22E571C2E4C2E5C2E6C2E7B400044A
:101ED60090000022B4010490000C22B40204900089
:101EE6001822B4030490002422B404049000302283
:101EF600B4050490003C2290004822E56C30E403CF
:101F0600C22822D22822E56A30E403C22922D22935
:101F160022056F121F24121F30900030F02290000D
:101F26002FE004B56F03756F012290002FE0B56FA7
:101F36000122400122F56F2220282290002FE0B4D2
:101F46000412121F75121D78E559F0A3E55AF0A385
:101F5600E55BF022B40203021F90021FDE121F751A
:101F6600121D78E0F559A3E0F55AA3E0F55B22E5EA
:101F76006FB4010490003622B4020490009922B492
:101F860003049000FC2290015F22E56FB4012390C8
:101F96000036121D78E559F0A3E55AF0A3E55BF08B
:101FA6009000FC121D78E559F0A3E55AF0A3E55B15
:101FB600F022B40222900099121D78E559F0A3E5AB
:101FC6005AF0A3E55BF090015F121D78E559F0A386
:101FD600E55AF0A3E55BF022900036121D78E5592C
:101FE600F0A3E55AF0A3E55BF0900099121D78E5A1
:101FF60059F0A3E55AF0A3E55BF09000FC121D78BA
:10200600E559F0A3E55AF0A3E55BF090015F121DD8
:1020160078E559F0A3E55AF0A3E55BF02220291EE6
:1020260090002FE0B4040E122058121D8BE55CF0D0
:10203600A3E568F022B402030220730220B1122045
:1020460058121D8BE0F9A3E0900032F0E9900031C0
:10205600F022E56FB401049001C222B4020490029A
:102066000422B403049002462290028822E56FB44B
:10207600011B9001C2121D8BE55CF0A3E568F09090
:102086000246121D8BE55CF0A3E568F022B4021A45
:10209600900204121D8BE55CF0A3E568F0900288BF
:1020A600121D8BE55CF0A3E568F0229001C2121DBB
:1020B6008BE55CF0A3E568F0900204121D8BE55CED
:1020C600F0A3E568F0900246121D8BE55CF0A3E5EF
:1020D60068F0900288121D8BE55CF0A3E568F0229B
:1020E600C2AF790C90001605A2121EC905A21220D5
:1020F600FAD2AF22E0A343D20205A2F0A375D252D0
:1021060075D2A2E5D220E0FB53D2FD05A2D9E52285
:10211600C2AF790C121EC905A290001605A21221A3
:102126002AD2AF2243D202438E20E0A353D2FD53DC
:102136008EDF05A2F0A305A2D9EA22C2AF790C7BF5
:1021460000121DC105A290001605A2122157D2AF9A
:1021560022EB9305A2F0A305A20BD9F522E56AF4BA
:1021660030E163E569F430E45D7405120CE41202B3
:1021760036120236120236120236120236120236B1
:10218600120236C2AF1221CD1221DF1221EF122127
:10219600FF12220F12221F12222F12223FD2AF123B
:1021A60002361202361202361202361202361202B5
:1021B6003612023612023612023612023612023671
:1021C60012023612023622790C7B0090257E05A279
:0E21D60090001605A212215722790C900016D7
:1021E40005A290000005A21220FA22790C90001694
:1021F40005A290000C05A21220FA22790C90001678
:1022040005A290001805A21220FA22790C9000165B
:1022140005A290002405A21220FA22790C9000163F
:1022240005A290003005A21220FA22790C90001623
:1022340005A290003C05A21220FA22790C90001607
:1022440005A290004805A21220FA22E627F52708E5
:1022540009E637F528782722C3E697F5270809E623
:1022640097F5287827228627872908098628872A28
:102274001222EF782C22862C08862D08862E0886BA
:102284002F872909872A1222927827792E227530DE
:10229400007531101222D41222A51222C8D531F4AD
:1022A40022C3E52E9529E52F952AE53094005001A7
:1022B40022E52E9529F52EE52F952AF52FE5309464
:1022C40000F53022B3E52733F527E52833F5282236
:1022D400C3E52C33F52CE52D33F52DE52E33F52E02
:1022E400E52F33F52FE53033F53022E5278529F046
:1022F400A4F52C85F02DE528852AF0A4F52E85F08B
:102304002FE5288529F0A4252DF52DE52E35F0F5AA
:102314002EE52F3400F52FE527852AF0A4252DF589
:102324002DE52E35F0F52EE52F3400F52F22B4F0EF
:102334000122400274F022B478012240027478220F
:10234400B43001224002743022900010E004B41032
:10235400027400F0900000A98229F582E022900026
:1023640014E0FA900011E004B40F0274FFF0902519
:102374005E932A900014F0900013E004B4100274E9
:1023840000F0F9900014E0FA900000E58229F5824B
:10239400EAF022900014E0FA900012E004B4110272
:1023A40074FFF090256D932A900014F012237B2281
:1023B40012234D5401600812234D541F24602274CB
:1023C4007F2212234D75F0058412234424302212F7
:1023D400234D5401600D12234D75F00584122344DE
:1023E40024302212234D75F00584122344246022E4
:1023F400E56B20E210D22430320FC282D287C2B6FB
:10240400D280C23222C224D232223009120542E5DD
:1024140042B4FF0B0543E543B4FF04C208C20922DA
:102424000540E540B4FF190541E541B4FF1275408C
:10243400FF7541FF753CFF753DFF85404885414967
:1024440022E56B30E103C20A22200A13D20A3009C2
:1024540006C20912253D22754200754300D20922A5
:10246400E56B30E003C20B22200B48D20B3024046E
:10247400C287D282E555240275F00284E5F0B400E7
:102484001885404885414975400075410085483CA0
:0E24940085493D85483E85493F754F00754E90
:1024A20000054D05551224B8D200D201302406127F
:1024B2001F3E02202322E555B4100E755500754DBE
:1024C20000302405C2A2121F1722E56B30E703C2B7
:1024D2000622200608D206D226D2B6C2A222E56A77
:1024E20030E703C20722200708D207D226D2B6C29B
:1024F200A2222024012220260122754000754100DB
:1025020085483C85493D85483E85493F755500755E
:102512004F00754E00754D00756F01C226223024A2
:10252200012220260122754200754300854A448516
:102532004B45754C00756F01C22622854232854398
:102542003375340075350078327536187537007971
:102552003612227A864A08E604F54B2203002C0C36
:1025620001057E2133E6FF0B4D68146405150D5AF3
:102572004B1B26351E1A96114042C8D50001020394
:102582000405060708090A0B008102830405860771
:1025920088098A0B008182830485860788898A8B51
:1025A200008182830485860788098A8B0081828361
:1025B2000485860788898A0B0081828304850687C1
:1025C20088898A0B008182838405868788890A8BA1
:1025D200008182030485860788090A8B0081020331
:1025E2008405860708898A0B008102038405860711
:1025F20008890A8B008182038485860788898A8BF1
:10260200008182038485860788098A8B0081820380
:102612008485860788890A8B0081820384850687E0
:1026220088890A8B008182038405060788890A8BC0
:10263200008102038405860788090A8B0001820350
:102642008405860708890A8B0081028304850607B0
:1026520088098A0B008102038405068708098A0B10
:10266200008102830405860788090A8B00810283A0
:102672000485068708890A8B008102838405860700
:1026820088890A8B000182830405860708890A8BE0
:10269200008102038405060708898A0B0001820370
:1026A2008485860708898A8B000182830405860750
:1026B20008898A0B008102830405860708890A8B30
:1026C200008102030485060708098A0B00018203C0
:1026D2000485060788090A8B464C414D4520544122
:1026E2004D45204D414348494E45204555524F20C6
:1026F2005241434B2056455253494F4E202D2032D2
:102702003031302056455253494F4E20312E303011
:0D27120020286329627920616D7065726571
:00000001FF
